:020000040000FA
:100000000128831687010430850010309F000430DA
:1000100091000130810080309000831232308500E1
:10002000870189309F00073099008B01AB01A30144
:10003000A401A001A101A201A7012815A530AA00D1
:100040001030A5000514851281010B1D25280B1108
:100050008516051087012F308700051281010B1DC1
:100060002F280B1105160510870105148510810135
:100070000B1D38280B11851405108701AA0B2228A7
:100080000830AA002008C120BC2087008512810109
:10009000A81C60289F149F184B28831603131E0862
:1000A00083120313A307031C5628A40A1E08A407DF
:1000B000A810A50B5E28A8151030A5000830AA00CE
:1000C0000B1D60280B118516051087012108C12022
:1000D000BC20870005128101A81D79280430A600E4
:1000E0000310A40CA30CB30CA60B7028A811B30129
:1000F00095200B1D79280B11051605108701AA0BF9
:100100008428A8140830AA000030A202031942284B
:100110002208C120BC208700851081010B1D8E287C
:100120000B11851405108701422803101030A70019
:10013000A001A101A30DA40DA00DA10DA70BAA283C
:1001400021080F39A200200E0F39A10020080F3915
:10015000A000080020308400B12021308400B120AC
:100160009A2803300007A600A61980003030000747
:10017000A600A61B80000034AB0005102B1B051445
:1001800008000F3982073F3409345E345B34693428
:100190007334773419347F347B34003400340034C2
:1001A000003400340034FF3FFF3FFF3FFF3FFF3F7D
:1001B000FF3FFF3FFF3FFF3FFF3FFF3FFF3FFF3F4F
:1001C000FF3FFF3FFF3FFF3FFF3FFF3FFF3FFF3F3F
:1001D000FF3FFF3FFF3FFF3FFF3FFF3FFF3FFF3F2F
:1001E000FF3FFF3FFF3FFF3FFF3FFF3FFF3FFF3F1F
:1007F000FF3FFF3FFF3FFF3FFF3FFF3FFF3F2034F3
:10420000FF00FF00FF00FF00FF00FF00FF00FF00B6
:10421000FF00FF00FF00FF00FF00FF00FF00FF00A6
:10422000FF00FF00FF00FF00FF00FF00FF00FF0096
:10423000FF00FF00FF00FF00FF00FF00FF00FF0086
:10424000FF00FF00FF00FF00FF00FF00FF00FF0076
:10425000FF00FF00FF00FF00FF00FF00FF00FF0066
:10426000FF00FF00FF00FF00FF00FF00FF00FF0056
:10427000FF00FF00FF00FF00FF00FF00FF00FF0046
:10428000FF00FF00FF00FF00FF00FF00FF00FF0036
:10429000FF00FF00FF00FF00FF00FF00FF00FF0026
:1042A000FF00FF00FF00FF00FF00FF00FF00FF0016
:1042B000FF00FF00FF00FF00FF00FF00FF00FF0006
:1042C000FF00FF00FF00FF00FF00FF00FF00FF00F6
:1042D000FF00FF00FF00FF00FF00FF00FF00FF00E6
:1042E000FF00FF00FF00FF00FF00FF00FF00FF00D6
:1042F000FF00FF00FF00FF00FF00FF00FF00FF00C6
:02400E0084012B
:08400000FF3FFF3FFF3FFF3FC0
:00000001FF
